S01E000062696E2F64656D6F70726F675F73746D3332673037312E737265632A
S31508002000009000205D260008AD260008AD260008D1
S3150800201000000000000000000000000000000000B2
S31508002020000000000000000000000000AD260008C7
S315080020300000000000000000AD2600086744000804
S31508002040AD260008AD260008AD260008AD26000816
S31508002050AD260008AD260008AD260008AD26000806
S31508002060AD260008AD260008AD260008AD260008F6
S31508002070AD260008AD260008AD260008AD260008E6
S31508002080AD260008AD260008AD260008AD260008D6
S31508002090AD260008AD260008AD260008AD260008C6
S315080020A0AD260008AD260008AD260008AD260008B6
S315080020B0AD260008AD260008AD260008EE11AA5583
S315080020C010B5064C2378002B07D1054B002B02D000
S315080020D0044800E000BF0123237010BD3804002027
S315080020E00000000024470008044B10B5002B03D05D
S315080020F00349044800E000BF10BDC04600000000C8
S315080021003C04002024470008002243088B4274D36D
S3150800211003098B425FD3030A8B4244D3030B8B42DA
S3150800212028D3030C8B420DD3FF22090212BA030CE3
S315080021308B4202D31212090265D0030B8B4219D3C4
S3150800214000E0090AC30B8B4201D3CB03C01A5241E4
S31508002150830B8B4201D38B03C01A5241430B8B422C
S3150800216001D34B03C01A5241030B8B4201D30B0315
S31508002170C01A5241C30A8B4201D3CB02C01A52413C
S31508002180830A8B4201D38B02C01A5241430A8B42FF
S3150800219001D34B02C01A5241030A8B4201D30B02E8
S315080021A0C01A5241CDD2C3098B4201D3CB01C01A02
S315080021B0524183098B4201D38B01C01A524143090C
S315080021C08B4201D34B01C01A524103098B4201D3FA
S315080021D00B01C01A5241C3088B4201D3CB00C01A67
S315080021E0524183088B4201D38B00C01A52414308DF
S315080021F08B4201D34B00C01A5241411A00D2014604
S31508002200524110467047FFE701B5002000F006F876
S3150800221002BDC0460029F7D076E770477047C0462A
S31508002220002B11D1002A0FD1002900D1002802D095
S315080022300021C943081C07B4024802A140180290AD
S3150800224003BDC046D9FFFFFF03B4684601B502982F
S3150800225000F006F8019B9E4602B00CBC7047C046CB
S31508002260F0B557464E464546DE46E0B5040083B00F
S315080022700D00924699468B4230D82DD04946504695
S3150800228000F0C0F829000600200000F0BBF8331A59
S315080022909846203B9B4633D45A465346934042467B
S315080022A01F00534693401E00AF423AD8AF4200D1B2
S315080022B07BE05B46A41BBD41002B00DA78E00022D8
S315080022C000230092019301235A4693400193012368
S315080022D042469340009328E08242CFD90022002349
S315080022E0009201930C9B002B01D01C605D60009846
S315080022F0019903B03CBC90469946A246AB46F0BD50
S31508002300424620239B1A5246DA40414613004A4663
S315080023108A40170042461F43534693401E00AF4269
S31508002320C4D900220023009201934346002BD9D03A
S31508002330FB079C46614672080A437B0846460EE040
S31508002340AB4201D1A2420CD8A41A9D4101202419FE
S315080023506D410021013E24184D41002E06D0AB42A6
S31508002360EED9013E24196D41002EF8D10098019945
S315080023705B4600196941002B25DB2B005A4644466B
S31508002380D3402A00E2401C005B461500002B2BDBDD
S3150800239026005F46BE40330026004746BE40320050
S315080023A0801A9941009001919CE7A342B9D880E729
S315080023B04246202300219B1A002200910192012205
S315080023C0DA40019283E7424620239B1A2A004646B2
S315080023D09A402300F340444613432A00E2401C0077
S315080023E05B461500002BD3DA2023424626009B1AAB
S315080023F0DE402F00B4464646B74066463B003343A8
S31508002400CAE7C04610B5002903D100F007F8203006
S3150800241002E0081C00F002F810BDC0461C2101238A
S315080024201B04984201D3000C10391B0A984201D3A9
S31508002430000A08391B09984201D30009043902A287
S31508002440105C40187047C0460403020201010101EE
S31508002450000000000000000070B50C4D0C4E761B05
S31508002460B61005D0002408CD01349847A642FAD103
S3150800247002F058F9074D084E761BB61005D0002411
S3150800248008CD01349847A642FAD170BDA84700087E
S31508002490A8470008A8470008B0470008F0B5050097
S315080024A083074AD0541E002A44D0CEB20300032222
S315080024B002E00135013C3DD301332E701342F8D1B9
S315080024C0032C2FD9FF220A40150215432A04154367
S315080024D00F2C35D92700103F3F093E01B4461E0090
S315080024E01A0010366644156055609560D56010323E
S315080024F0B242F8D10F260C2201373F012640DB19DC
S315080025003700224217D03E1FB608B400A4461A0068
S315080025101C1D644420C2A242FCD103240136B60025
S315080025209B193C40002C05D0C9B21C1919700133FF
S315080025309C42FBD1F0BD3400F4E714000300BFE76A
S315080025402700E0E7034B10B5002B02D0024800F045
S3150800255005F810BD000000006D25000810B5010043
S3150800256000230022002000F019F810BD70B5074DB1
S31508002570074C641BA41005D0013CA300EB589847F0
S31508002580002CF9D102F0D4F870BDC046B047000857
S31508002590B44700087047C0467047C046F0B5DE46E7
S315080025A045464E465746E0B52A4C83B00500206896
S315080025B090469B460E00FFF7EDFF274B1B680193DD
S315080025C0A423019A5B00D258002A38D053682068A1
S315080025D01F2B3ADC002D0ED1591C02339B0051608B
S315080025E09E50FFF7D9FF002003B03CBC90469946A1
S315080025F0A246AB46F0BD99008946914441468824D7
S315080026004F463951C4214900884690444146873C83
S315080026109C400968A24621438C46414664460C60A4
S3150800262084214C465F4649006750022DD4D11100DB
S3150800263055468D31FF310C6825430D60CCE7019A6C
S3150800264001994D32FF32CA50C0E7FFF7A5FF0120B6
S315080026504042C9E7280400203C4700080D48854643
S31508002660002103E00C4B5B58435004310B480C4BDC
S3150800267042189A42F6D30B4A02E00023136004324A
S31508002680094B9A42F9D300F013F8FFF7E5FE01F07B
S3150800269021FFFEE700900020B44700080000002054
S315080026A0380400203804002058050020FEE7000002
S315080026B0024B802212059A607047C04600ED00E082
S315080026C010B5144A136814490B400343136080225B
S315080026D092000023904201D0180010BD0F4B1B68D2
S315080026E05800C01840000E49FFF70EFD0130094B8F
S315080026F05B695B050AD507498022D20001384B6918
S31508002700134205D00028F9D10323E5E70023E3E7C0
S315080027100023E1E700700040FFF9FFFF2C040020CA
S3150800272040420F00F0B5CE46474680B583B0041E3A
S3150800273000D149E20368DB0738D5C74A91683823D0
S315080027400B40D268102B26D0082B27D0636880222E
S31508002750520293427BD0A022D20293427ED0BE4B35
S315080027601A68BE490A401A601A68BD490A401A60C2
S315080027706368002B7ED001F02FFD0700B64E80253A
S31508002780AD0233682B4211D101F026FDC01B642827
S31508002790F7D9032019E2D2439307D7D1AE4B1B686A
S315080027A09B0303D56368002B00D113E223689B07BC
S315080027B02BD5A94A916838230B40D268102B69D0CB
S315080027C0002B6CD1A44B1B685B0500D525E2A249FA
S315080027D04A6863691B02A348024013434B609E4A3A
S315080027E01368A1490B4021690B43136013689B04C6
S315080027F05B0F9E4ADA4013009D4A13609D4B18688A
S3150800280001F0A2FC002800D0E6E123681B0700D4EB
S315080028108BE0914B9A6838231340182B7DD0A36917
S31508002820002B00D1C3E08C4A136E01210B431366BB
S3150800283001F0D2FC0700884E0225336E1D4274D182
S3150800284001F0CAFCC01B0228F7D90320BDE1824A61
S31508002850116880235B020B43136089E77E4B196876
S315080028608022D2020A431A601968802252020A4359
S315080028701A607DE701F0B0FC0700774E8025AD02AF
S3150800288033682B4292D001F0A7FCC01B6428F7D905
S3150800289003209AE10D3B1340022B00D1A4E1E36823
S315080028A0002B24D06C4A13686F490B4021690B43EF
S315080028B01360116880235B000B43136001F08CFCE6
S315080028C00700654E8025ED0033682B4206D101F0DE
S315080028D083FCC01B0228F7D9032076E15E494A68C3
S315080028E063691B025F48024013434B608DE75A4AEF
S315080028F0136861490B40136001F06EFC0700564EE1
S315080029008025ED0033682B4200D17EE701F064FC98
S31508002910C01B0228F6D9032057E14F4B1B6E9B07B5
S3150800292003D5A369002B00D158E123685B0700D4BF
S31508002930ABE0494B9A6838231340202B4BD0464BC3
S31508002940DB6B00229046DB000BD4434AD16B802018
S3150800295040050143D163D36B03400193019B0123D7
S315080029609846464B1B68DB053ED5A368012B51D01C
S31508002970052B55D0384BDA6D01218A43DA65DA6DB5
S3150800298003318A43DA65A368002B53D001F024FC8F
S315080029908146314F02263A4DFB6D1E4272D101F037
S315080029A01BFC4B46C01AA842F6D903200DE12A4A59
S315080029B0136E01218B43136601F00EFC0700264EA9
S315080029C00225336E1D42B0D001F006FCC01B02285A
S315080029D0F7D90320F9E0204BDB6D9B0755D5A36893
S315080029E0002B52D10120F0E0244A116880235B00B5
S315080029F00B43136001F0F0FB0500204F802676009C
S31508002A003B683342B1D101F0E7FB401B0228F7D9F6
S31508002A100320DAE0104AD36D01210B43D365B2E7F0
S31508002A200D4BDA6D04210A43DA65DA6D03390A4378
S31508002A30DA65A8E701F0D0FB8146074F0226104D5C
S31508002A40FB6D1E421ED001F0C7FB4B46C01AA842BA
S31508002A50F6D90320B9E0C04600100240FFFFFEFF8A
S31508002A60FFFFFBFFFF80FFFFFFC7FFFF0024F40007
S31508002A702C04002034040020FFFEFFFF00700040F5
S31508002A80881300004346012B29D0E3690020002B58
S31508002A9000D19AE0674A916838220A40102A69D01C
S31508002AA0022B22D0634B1A6863490A401A60DA6817
S31508002AB003218A43DA60DA6860490A40DA6001F07D
S31508002AC08BFB06005B4D8024A4042B6823424FD061
S31508002AD001F082FB801B0228F7D9032075E0554ACE
S31508002AE0D36B57490B40D363CFE7524A1368524911
S31508002AF00B40136001F070FB07004E4E8025AD04B5
S31508002B0033682B4206D001F067FBC01B0228F7D9B1
S31508002B1003205AE0474AD168236A606A0343494852
S31508002B2001400B43E16A0B43216B0B43616B0B437B
S31508002B30A16A09020B43D360116880235B040B4327
S31508002B401360D16880235B050B43D36001F044FB17
S31508002B500600384D8024A4042B68234206D101F0D0
S31508002B603BFB801B0228F7D903202EE000202CE02F
S31508002B7000202AE0012B33D02E4BDA6803231340BA
S31508002B800120216A8B4220D170231340616A8B424F
S31508002B901BD1FE21C9011140A36A1B02994214D117
S31508002BA0F8239B031340E16A8B420ED1E0231B05F1
S31508002BB01340216B8B4208D1500F4007636BC01A34
S31508002BC0431E9841C0B200E0012003B00CBC9046F9
S31508002BD09946F0BD0120F8E70120F6E70120F4E761
S31508002BE00120F2E70120F0E7124B1B685B0508D4C9
S31508002BF010494A6863691B021348024013434B6035
S31508002C00FCE5E368002BEDD00A494A6863691B02B4
S31508002C100D48024013434B60F0E50120E368002BA2
S31508002C20D3D004494A6863691B0207480240134324
S31508002C304B60D4E500100240FFFFFFFEFFFFFEEEEB
S31508002C40FFFFFFEF8C80C111FF80FFFF10B5274BF8
S31508002C509B6838221A4206D1244B1B689B045B0FDB
S31508002C602348D84010BD214B9A6838231340082BB7
S31508002C7037D01E4B9A6838231340102B11D01B4BA4
S31508002C809A6838231340202B2DD0184B9B68382080
S31508002C9018401838434258414042FA23DB0118408D
S31508002CA0E0E7124AD368D1684906490F0131DB4388
S31508002CB09B070ED00D4BD8684004440E0C48FFF70E
S31508002CC023FA6043094BD968490F0131FFF71CFA0B
S31508002CD0C8E7D0684004440E0648FFF715FA604373
S31508002CE0F0E70448BEE780200002BBE70010024078
S31508002CF00024F40000127A00F8B5CE46474680B59F
S31508002D0004000D00002800D1B3E05C4B1A680723C5
S31508002D1013408B4221D323689A070ED55B0705D546
S31508002D20574A9168E023DB010B439360544A936842
S31508002D3054490B40A1680B4393602368DB0759D5B8
S31508002D406368012B22D0022B40D0002B44D14C4A79
S31508002D50126852051FD401206EE0484A13680721FD
S31508002D608B432B43136001F037FA8146434F0726FE
S31508002D70454B98463B683340AB42CCD001F02CFA21
S31508002D804B46C01A4045F5D9032055E03C4A12681F
S31508002D90920300D46FE03A498A68072082431343B6
S31508002DA08B6001F019FA8146354F3826364B98461E
S31508002DB0BA6832406368DB009A421BD001F00CFA0D
S31508002DC04B46C01A4045F3D9032035E02C4A126811
S31508002DD09201E0D401202FE0032B05D0284AD26DBA
S31508002DE09207D8D4012027E0254A126E9207D2D43A
S31508002DF0012021E0214B1A6807231340AB421FD854
S31508002E0023685B0706D51E4A936820490B40E1688C
S31508002E100B439360FFF71AFF194B9B681B051B0FA3
S31508002E209B001B4A9B581F221340D840194B186019
S31508002E30194B186801F088F90CBC90469946F8BDFC
S31508002E400E4A136807218B432B43136001F0C4F91C
S31508002E5081460A4F07260C4B98463B683340AB42DF
S31508002E60CED001F0B9F94B46C01A4045F5D9032032
S31508002E70E2E70120E0E70120DEE7C0460020024045
S31508002E8000100240FFF0FFFF88130000FF8FFFFFCE
S31508002E90404700082C04002034040020014B186821
S31508002EA07047C0462C040020064B9B685B045B0FEA
S31508002EB09B00054A9B581F221340044A1068D840B5
S31508002EC07047C04600100240804700082C040020C6
S31508002ED070B5002814DB8408A400144B9C4664448F
S31508002EE0C026B600A55903221040C000FF231A00C9
S31508002EF08240954389010B4083401D43A55170BD0F
S31508002F00C0B20F220240083A92089200084BD31822
S31508002F10DD6903242040C000FF2214008440A54335
S31508002F2089010A4082402A43DA61E8E700E100E0C5
S31508002F3000ED00E001380A4B98420FD8094A506064
S31508002F400948036A1B021B0AC02109060B430362D0
S31508002F500023936007331360002070470120FCE7C5
S31508002F60FFFFFF0010E000E000ED00E0042805D0B8
S31508002F70054A136804218B4313607047024A136895
S31508002F8004210B431360F8E710E000E0704710B522
S31508002F90FFF7FCFF10BD0000F0B5DE4657464E466B
S31508002FA04546E0B583B00A68002A00D1B3E000239D
S31508002FB00124A0460F34A2460D3CA1468024640590
S31508002FC0A346584C041965426C41644201943CE09E
S31508002FD0DC08A4000419276A07251D40AD000F2246
S31508002FE0AA4097430A69AA4015003D43256236E080
S31508002FF00025B5403D4325664B4D80242C59009A43
S31508003000D5434A68D2037AD42C40474E8027F451D8
S31508003010842434594A68920374D42C40424E842737
S31508003020F45134684A68D2026FD42C403E4E34605C
S3150800303074684A6892026BD422002A403A4C62604D
S3150800304001330A681400DC4065D046469E4032408B
S315080030500092F5D04C685546AC43022CB8D00468AB
S315080030605F004D46BD40ED432C40A4464C684A4699
S315080030701440BC406246144304604C68524694436C
S31508003080013C012C11D884682C40A446CC68BC406D
S315080030906246144384604468B44326004A681409A7
S315080030A0424614409C4034434460C4682C408D68B2
S315080030B0BD402543C5604A685C462242C0D09C088C
S315080030C0A400194A94466444256E4E461E40F600EE
S315080030D00F27B740BD432F00A025ED05A84287D08E
S315080030E0124DA84207D0124DA84206D0019D42466D
S315080030F0954305357DE701257BE7022579E7009AA3
S31508003100144382E7009A144388E7009A14438DE72C
S31508003110009A224392E703B03CBC90469946A246E1
S31508003120AB46F0BD00F4FFAF0018024000040050A3
S3150800313000080050002A01D0816170478162FCE7CF
S3150800314070470000F8B504000168836802691343F4
S3150800315042691343C26913430A68406E0343CE4863
S31508003160024013430B6022685368CC490B40E16860
S315080031700B435360A1692268C94B9A4201D0236A5E
S3150800318019439368C74803400B4393602268D36A80
S315080031900F218B43616A0B43D3622268C24B9A4262
S315080031A05FD0C24B9A4200D1B8E0C14B9A4201D1D6
S315080031B000F0D6FDBF4B9A4201D100F0D4FDB849C4
S315080031C010238A4262D1BC4B5B6DC02109010B40BA
S315080031D08021C9008B4200D131E100D8D9E0802294
S315080031E01201934200D1F5E0C02212010120934258
S315080031F001D000F025FC636A002B01D100F07BFDAD
S31508003200012B01D100F07BFD022B01D100F07BFDE3
S31508003210032B01D100F07BFD042B01D100F07AFDD0
S31508003220052B01D100F07AFD062B01D100F079FDBE
S31508003230072B01D100F078FD082B01D100F078FDAD
S31508003240092B01D100F078FD0A2B01D100F078FD99
S315080032500B2B01D100F078FD082580231B0200F016
S31508003260EAFC954B596D03230B40012B01D100F065
S315080032706EFD002B69D0022B01D100F06BFD033BDC
S315080032805A4253415B42072293431033802212026B
S31508003290E169914200D150E2022B01D100F01CFCF9
S315080032A000D8A2E3042B01D100F056FC082B00D06D
S315080032B0CFE3636A002B01D100F08CFC012B01D10E
S315080032C000F094FC022B01D100F093FC032B01D1F2
S315080032D000F092FC042B01D100F090FC052B01D1E3
S315080032E000F08FFC062B01D100F08DFC072B01D1D5
S315080032F000F08BFC082B01D100F08AFC092B01D1C8
S3150800330000F089FC0A2B01D100F088FC0B2B01D1B7
S3150800331000F087FC80231B0200F05EFC664B5B6DA9
S315080033200C211940042901D100F017FD0AD90223FE
S315080033300829ABD00C394B424B415B4207229343D9
S315080033401033A3E710230029A0D1554B9A4201D088
S3150800335000F00CFDFFF7A8FD636A0121002B1DD0C4
S31508003360012B1AD0022B23D0032B23D0042B23D0D6
S31508003370052B23D0062B23D0072B23D0082B23D0AD
S31508003380092B23D00A2B23D00B2B07D180214900E8
S3150800339004E00120002BD8D052E30221FEF7B4FE48
S315080033A0030000250020002B00D149E300F043FC70
S315080033B00421F3E70621F1E70821EFE70A21EDE703
S315080033C00C21EBE71021E9E72021E7E74021E5E7B3
S315080033D08021E3E7636A002B01D100F02AFC012B68
S315080033E001D100F067FC022B01D100F066FC032B2B
S315080033F001D100F065FC042B01D100F064FC052B1B
S3150800340001D100F063FC062B01D100F062FC072B0A
S3150800341001D100F061FC082B01D100F060FC092BFA
S3150800342001D100F05FFC0A2B01D100F05EFC0B2BEA
S3150800343001D100F05DFC0225204B00F0FCFBFFF7F4
S3150800344005FC636A0121002B19D0012B16D0022B2B
S315080034501AD0032B1AD0042B1AD0052B1AD0062BF8
S315080034602ED0072B2ED0082B2ED0092B2ED00A2B88
S315080034702ED00B2B03D18021490000E00221FEF754
S3150800348043FE030004258DE70421F8E70621F6E745
S315080034900821F4E70A21F2E7F369FFCFFFCFFFFF20
S315080034A000800040FFF4FF1100380140004400404E
S315080034B000480040004C0040001002400024F40080
S315080034C00C21DCE71021DAE72021D8E74021D6E7EE
S315080034D08021D4E70022002D22D1FFF7E5FC636A9C
S315080034E001260027002B26D0012B22D0022B37D00D
S315080034F0032B38D0042B39D0052B3AD0062B3BD0DA
S31508003500072B3CD0082B3DD0092B3ED00A2B3FD0A9
S315080035100B2B10D18026760000270CE00120002214
S31508003520B249B34BD3188B4200D97CE32368DA60DF
S3150800353086E202260027656832003B000021FEF776
S315080035406FFE060E0B02334302026808002180183C
S3150800355059412A000023FEF763FE02000020DFE738
S3150800356004260027E7E706260027E4E708260027BB
S31508003570E1E70A260027DEE70C260027DBE7102608
S315080035800027D8E720260027D5E740260027D2E7D8
S3150800359080260027CFE7636A002B18D0012B22D09C
S315080035A0022B23D0032B24D0042B25D0052B26D081
S315080035B0062B27D0072B28D0082B29D0092B2AD051
S315080035C00A2B2BD00B2B2CD08A4E002701E0894ED4
S315080035D0002750080021801979410023FEF720FEB4
S315080035E0020000209CE7844E0027F2E7834E00275E
S315080035F0EFE7834E0027ECE7824E0027E9E7824E85
S315080036000027E6E7814E0027E3E7814E0027E0E73B
S31508003610804E0027DDE7804E0027DAE77F4E002739
S31508003620D7E77F4E0027D4E7FFF710FB636A01262A
S315080036300027002B1BD0012B17D0022B2CD0032BD5
S315080036402DD0042B2ED0052B2FD0062B30D0072BB0
S3150800365031D0082B32D0092B33D00A2B34D00B2B80
S3150800366005D180267600002701E002260027656836
S3150800367032003B000021FEF7D3FD060E0B02334352
S31508003680020268080021801859412A000023FEF723
S31508003690C7FD0200002043E704260027E7E70626C1
S315080036A00027E4E708260027E1E70A260027DEE7E1
S315080036B00C260027DBE710260027D8E72026002758
S315080036C0D5E740260027D2E780260027CFE78026C1
S315080036D03604002750080021801979410023FEF797
S315080036E09FFD020000201BE78026F6030027F1E76E
S315080036F08026B6030027EDE74A4E0027EAE780262C
S3150800370076030027E6E7484E0027E3E7474E0027FB
S31508003710E0E7802636030027DCE78026F602002746
S31508003720D8E78026B6020027D4E780267602002747
S31508003730D0E7802636020027CCE7022B00D1AEE080
S3150800374032D9042B00D1EAE0082B00D084E0636A62
S31508003750002B00D122E1012B00D12BE1022B00D155
S315080037602BE1032B00D12BE1042B00D12AE1052BF9
S3150800377000D12AE1062B00D129E1072B00D128E147
S31508003780082B00D128E1092B00D128E10A2B00D10A
S3150800379028E10B3B584258414042254B18408023AC
S315080037A05B029C466044FBE0002B43D1FFF77CFBA1
S315080037B0636A0121002B53D0012B50D0022B5CD019
S315080037C0032B5CD0042B5CD0052B5CD0062B5CD07D
S315080037D0072B5CD0082B5CD0092B5CD00A2B5CD05D
S315080037E00B2B3DD1802149003AE0C046FFFC0F0073
S315080037F000FDFFFF000024F40000127A0000093DD6
S3150800380000AAB0280080841E00006A1800555814C3
S315080038100040420F0020A1070090D0030048E801AD
S315080038200024F4000055150000CC0C0000AA0A007C
S315080038300001FFFF0120002397491A00103A8A4227
S3150800384000D9F2E10F22190091430A0021681B07EB
S315080038505B0F1343CB60F3E001200023ECE7022162
S315080038606568FEF751FC40006B08C0182900FEF792
S315080038704BFC03041B0C0020DEE70421F0E70621BD
S31508003880EEE70821ECE70A21EAE70C21E8E7102130
S31508003890E6E72021E4E74021E2E78021E0E7636AE2
S315080038A0002B1DD0012B26D0022B26D0032B26D089
S315080038B0042B26D0052B26D0062B26D0072B26D060
S315080038C0082B26D0092B26D00A2B26D00B3B58428C
S315080038D058414042714B1840714B9C46604400E089
S315080038E06F4863685B0818186168FEF70DFC0304E7
S315080038F01B0C0020A0E76B48F3E76B48F1E76B4821
S31508003900EFE76B48EDE76B48EBE76B48E9E76B4891
S31508003910E7E76B48E5E76B48E3E76B48E1E7FFF75E
S3150800392095F9636A0121002B19D0012B16D0022BB9
S3150800393022D0032B22D0042B22D0052B22D0062BF3
S3150800394022D0072B22D0082B22D0092B22D00A2BD3
S3150800395022D00B2B03D18021490000E002216568A3
S31508003960FEF7D2FB40006B08C0182900FEF7CCFB17
S3150800397003041B0C00205FE70421F0E70621EEE7AD
S315080039800821ECE70A21EAE70C21E8E71021E6E737
S315080039902021E4E74021E2E78021E0E78020400299
S315080039A063685B0818186168FEF7AEFB03041B0C16
S315080039B0002041E780200002F2E78020C001EFE7FF
S315080039C04248EDE780208001EAE74148E8E74148B8
S315080039D0E6E780204001E3E780200001E0E7802059
S315080039E0C000DDE780208000DAE7002B1ED1FFF754
S315080039F05BFA636A0121002B2FD0012B2CD0022BF6
S31508003A0037D0032B37D0042B37D0052B37D0062BCE
S31508003A1037D0072B37D0082B37D0092B37D00A2BAE
S31508003A2037D00B2B19D18021490016E0012000233D
S31508003A3019491A00103A8A4200D9F8E02268D36078
S31508003A4001236A22A352023AA3520023E36623679C
S31508003A50F8BD01200023EBE702216568FEF754FB59
S31508003A606B08C0182900FEF74FFB03041B0C002047
S31508003A70DEE70421F1E70621EFE70821EDE70A2151
S31508003A80EBE70C21E9E71021E7E72021E5E74021EC
S31508003A90E3E78021E1E7C046EFFF000048A019FEF2
S31508003AA00048E8010024F40000127A00546151002D
S31508003AB000093D0000D43000AAB0280080841E000A
S31508003AC040420F0020A1070090D00300AA2A000058
S31508003AD09819000054150000636A002B1DD0012BAD
S31508003AE026D0022B26D0032B26D0042B26D0052B36
S31508003AF026D0062B26D0072B26D0082B26D0092B16
S31508003B0026D00A2B26D00B3B5842584140429C4BA4
S31508003B1018409C4B9C46604400E09A4863685B08E2
S31508003B2018186168FEF7F0FA03041B0C00207FE7FB
S31508003B309548F3E79548F1E79548EFE79548EDE7A7
S31508003B409548EBE79548E9E79548E7E79548E5E7B7
S31508003B509548E3E79548E1E7FFF778F8636A0121B6
S31508003B60002B19D0012B16D0022B21D0032B21D0E4
S31508003B70042B21D0052B21D0062B21D0072B21D0B1
S31508003B80082B21D0092B21D00A2B21D00B2B03D1AE
S31508003B908021490000E002216568FEF7B5FA6B0846
S31508003BA0C0182900FEF7B0FA03041B0C00203FE7F3
S31508003BB00421F1E70621EFE70821EDE70A21EBE703
S31508003BC00C21E9E71021E7E72021E5E74021E3E7B3
S31508003BD08021E1E780231B0262685008C0181100A3
S31508003BE0FEF792FA03041B0C002021E78023DB0171
S31508003BF0F2E780239B01EFE76D4BEDE780235B013E
S31508003C00EAE76C4BE8E76C4BE6E780231B01E3E742
S31508003C108023DB00E0E780239B00DDE780235B0051
S31508003C20DAE78023D8E701200AE7012008E7012020
S31508003C3006E70225534B626851008918012099420C
S31508003C4000D9FDE61103994200D2F9E6022D00D10A
S31508003C50A1E400D83EE4042D00D1E5E4082D00D007
S31508003C605CE4636A002B00D131E5012B00D13BE50A
S31508003C70022B00D13CE5032B00D13DE5042B00D1F6
S31508003C803DE5052B00D13EE5062B00D13EE5072B89
S31508003C9000D13EE5082B00D13FE5092B00D140E5D0
S31508003CA00A2B00D141E50B2B00D142E580263604CC
S31508003CB000270FE50225344BBDE70225334BBAE74B
S31508003CC00225334BB7E70225324BB4E70225324BC0
S31508003CD0B1E70225314BAEE70225314BABE70225AA
S31508003CE0304BA8E70225304BA5E702252F4BA2E764
S31508003CF00225324B9FE7082580231B029BE70825F0
S31508003D008023DB0197E7082580239B0193E7082595
S31508003D10274B90E7082580235B018CE70825254B70
S31508003D2089E70825244B86E7082580231B0182E7B7
S31508003D3008258023DB007EE7082580239B007AE799
S31508003D40082580235B0076E70825802373E704238C
S31508003D50FFF79CFA0223FFF799FA0423FFF796FA6E
S31508003D600023FFF793FA0023FFF790FA80231B023C
S31508003D70E2699A4200D119E50023FFF78DFAC04699
S31508003D8024D00CFF0024F40000127A0000093D003C
S31508003D90AAB0280080841E00006A1800555814002E
S31508003DA040420F0020A1070090D0030048E8010018
S31508003DB055150000CC0C0000AA0A000024F40000E7
S31508003DC0836ADB0706D5026853682C490B40C16A2B
S31508003DD00B435360836A9B0706D5026853682849D4
S31508003DE00B40016B0B435360836A5B0706D5026879
S31508003DF0536824490B40416B0B435360836A1B0786
S31508003E0006D50268536820490B40816B0B43536003
S31508003E10836ADB0606D5026893681C490B40C16BAA
S31508003E200B439360836A9B0606D502689368184914
S31508003E300B40016C0B439360836A5B060BD50268E3
S31508003E40536814490B40416C0B43536080235B0352
S31508003E50426C9A420AD0836A1B0606D502685368E2
S31508003E600D490B40C16C0B43536070470268536899
S31508003E700A490B40816C0B435360ECE7FFFFFDFFDB
S31508003E80FFFFFEFFFFFFFBFFFF7FFFFFFFEFFFFFC9
S31508003E90FFDFFFFFFFFFEFFFFFFFF7FFFFFF9FFFBC
S31508003EA0F0B5C64600B507000C0016009846069DF4
S31508003EB03A68D36923401B1B59424B41B3421ED172
S31508003EC06B1CF6D000F088F94346C01AA84201D800
S31508003ED0002DEDD13A6813680B490B4013603A6818
S31508003EE09368A331FF318B43936020238022BB5014
S31508003EF00432BB505C330022FA54032000E0002051
S31508003F0004BC9046F0BDC0465FFEFFFFF0B5CE4646
S31508003F10474680B585B004000D00170098468423EF
S31508003F20C358202B00D08FE0002900D192E0002A48
S31508003F3000D191E080235B0182689A4222D07C23DB
S31508003F40E35C012B00D189E07C230122E2540C3387
S31508003F500022E250043B2232E25000F03DF9039081
S31508003F605C23E7520233E752A36880225201934248
S31508003F700FD0002B22D12369002B1BD16033FF22DF
S31508003F80E25222E00369002BD9D1CB07D7D501200D
S31508003F905BE02369002B06D1324B6022A352994677
S31508003FA02E00002515E06023FF22E2529F33994632
S31508003FB000260EE060237F22E25206E080225205A8
S31508003FC093420DD060230022E2526023E35A9946B9
S31508003FD000265E23E35A9BB2002B2DD05E2718E0FD
S31508003FE02369002B03D160337F22E252EDE7602379
S31508003FF03F22E252E9E723685B6A4A461340338068
S315080040000236E35B013B9BB2E353E35B9BB2002BB7
S3150800401012D043460093039B002220212000FFF77D
S315080040203FFF00281CD1002DE5D023685B6A4A466D
S3150800403013402B700135E4E784232022E250083B25
S315080040400022E254002000E0022005B00CBC904695
S315080040509946F0BD0120F8E70120F6E70220F4E7CB
S315080040600320F2E7FF01000030B583B0040088237F
S315080040700022C25000F0B0F8050023681B681B0731
S315080040800ED423681B685B0717D420238022A3500D
S315080040900432A3505C330022E254002003B030BD42
S315080040A080210C4B00930300002289032000FFF7B0
S315080040B0F7FE0028E5D00320F0E78021054B0093A2
S315080040C02B000022C9032000FFF7EAFE0028DCD0F7
S315080040D00320E3E7FFFFFF0110B5041E30D080235D
S315080040E0C358002B22D080232422E250226813686A
S315080040F001218B4313602000FFF724F8012814D010
S31508004100A36A002B18D1226853680E490B405360E6
S31508004110226893682A218B43936022681368293999
S315080041200B4313602000FFF79FFF10BD7C3300226E
S31508004130C254FFF705F8D6E72000FFF741FEE2E78D
S315080041400120F2E7FFB7FFFF10B504000F4B19680F
S315080041500120002900D110BDFA208000FDF7D4FF08
S3150800416001000B4B1868FDF7CFFFFEF7E3FE0300CF
S315080041700120002BEFD1032CEDD80022210040426C
S31508004180FEF7A6FE034B1C600020E4E7300400207F
S315080041902C0400203404002010B5084A1168802336
S315080041A05B000B4313600020FFF7CEFF041E02D00E
S315080041B00124200010BD00F0EBF9FAE700200240C8
S315080041C0034A1368034909685B1813607047C046B9
S315080041D05405002030040020014B18687047C0467B
S315080041E054050020F0B5CE46474680B583B0040096
S315080041F0002023689B032BD5824BDB6B002290465D
S31508004200DB000BD47F4AD16B802040050143D16384
S31508004210D36B03400193019B012398467A4A1168A0
S3150800422080235B000B431360FFF7D6FF0700764E2B
S3150800423080256D0033682B4200D0D4E0FFF7CCFF11
S31508004240C01B0228F6D903204346012B00D1AAE059
S315080042502368DB0706D56B4A536D03218B436168D8
S315080042600B43536523689B0706D5664A536D0C2195
S315080042708B43A1680B43536523689B0606D5614AA1
S31508004280536D62490B40E1680B43536523689B05F0
S3150800429006D55C4A536D5E490B40A1690B435365CD
S315080042A023685B0506D5574A536D5A490B40E169A1
S315080042B00B43536523685B0606D5524A536D564928
S315080042C00B4021690B43536523685B040BD54D4AA4
S315080042D0536D9B009B08216A0B4353658023DB05BE
S315080042E0226A9A4265D023681B0306D5454A536D50
S315080042F040218B43616A0B43536523689B020BD5A8
S31508004300404A536D45490B40A16A0B4353658023C8
S31508004310DB03A26A9A4253D023685B020BD5394A5B
S31508004320536D3F490B40E16A0B43536580235B0499
S31508004330E26A9A424BD023681B050BD5314A536D66
S3150800434038490B4061690B4353658023DB01626979
S315080043509A4241D003B00CBC90469946F0BD226BF8
S315080043609A4246D0274BD86D2F4A0240DD6D8021F0
S3150800437049022943D965D96D2C4D2940D965DA6595
S31508004380C30736D5FFF728FF81461E4E0225284F5C
S31508004390F36D1D422DD1FFF71FFF4B46C01AB842D9
S315080043A0F6D9032050E7174AD36B22490B40D3634B
S315080043B04EE7144AD16880235B020B43D36092E729
S315080043C0104AD16880235B040B43D360A4E70D4AE7
S315080043D0D1680B43D360AEE70A4AD16880235B02F3
S315080043E00B43D360B6E7074BDB6DC0229200134040
S315080043F0B5D1044AD36D0C490B40216B0B43D365E9
S31508004400002021E70010024000700040FFF3FFFF84
S31508004410FFFFF3FFFFFFCFFFFFCFFFFFFFFFBFFF4A
S31508004420FFFFFFFEFF3FFFFFFFFCFFFFFFFFFEFF53
S3150800443088130000FFFFFFEF10B5FEF72FFDFA21E6
S315080044408900FDF761FEFEF775FD0420FEF78EFD77
S315080044500120002200214042FEF73AFD10BD10B5AA
S31508004460FFF7BAFE10BD10B5FFF7AAFEFEF78FFDDF
S3150800447010BD10B5A02000222021C005FEF75AFE67
S3150800448010BD000010B5FFF7EAFF04000F4B1B68CC
S31508004490C31AF422FF3293420ED90D4B1B78002B18
S315080044A00BD10B4BF33AFF3A1A70A0202021C00516
S315080044B0FEF740FE054B1C6010BD054B00221A7026
S315080044C0A0202021C005FEF735FEF3E7580400209A
S315080044D05404002000B5A1B02B4A2C4B9A60FFF774
S315080044E05BFE3822002112A8FDF7D8FF1022002112
S315080044F001A8FDF7D3FF3422002105A8FDF7CEFF5A
S3150800450080208000FEF7DCF80223129380225200F6
S315080045101592002216924032179219931A932E3347
S315080045201B931C9280239B021D9380239B041E933E
S31508004530C023DB051F9312A8FEF7F4F8002800D065
S31508004540FEE70723019302210291002303930493B4
S3150800455001A8FEF7D1FB002800D0FEE70223059349
S315080045600023079305A8FFF73DFE002800D0FEE7C5
S31508004570FFF762FFFFF77DFF00F05AF8FFF782FFAB
S3150800458000F07EF8FAE7C0460020000800ED00E0DB
S31508004590F0B58BB0254B1A6C012422431A641A6CA9
S315080045A022400192019A5A6B22435A635A6B22405F
S315080045B00292029A5A6B022632435A635A6B324067
S315080045C00392039ADA6B802189020A43DA63DB6B6A
S315080045D00B400493049B0520002200214042FEF76D
S315080045E077FC0220002200214042FEF771FC0120E0
S315080045F0002200214042FEF76BFC20230593069417
S31508004600002507950895A027FF0505A93800FEF798
S31508004610C3FC0C230593069607950895099405A9E6
S315080046203800FEF7B9FC0BB0F0BDC04600100240DA
S3150800463010B50A480A4B0360E1231B0243600023B6
S315080046408360C360036183610C224261C361802277
S31508004650120102624362FFF73FFD10BD5C040020B1
S3150800466000440040BFF34F8F034B044ADA60BFF3A0
S315080046704F8FC046FDE7C04600ED00E00400FA058E
S3150800468010B5234B1B78002B17D10122214922484C
S31508004690FFF73CFC002800D010BD1E4B1B78013BE1
S315080046A03F2BF9D8FFF7DBFE1C4B1860184B01228D
S315080046B01A701B4B00221A70EEE7194B1B78013350
S315080046C01449C918002301221348FFF71FFC0028C4
S315080046D013D1134A13780133DBB213700D4A1278DB
S315080046E09A42D9D10A4A002111700A4A5278FF2AF9
S315080046F0D2D1022BD0D1FFF7B5FFFFF7B0FE074B9B
S315080047001B6864339842C7D9014B00221A70C3E765
S3150800471029050020E80400205C0400202C05002060
S315080047202A050020F8B5C046F8BC08BC9E46704766
S31108004730F8B5C046F8BC08BC9E467047A9
S3150800473C000000200000000000000000000000003F
S3150800474C000000000000000000000000000000004F
S3150800475C0000000001000000020000000300000039
S3150800476C0400000006000000070000000800000016
S3150800477C0900000000000000000000000000000016
S3150800478C0000000001000000020000000300000009
S3090800479C0400000007
S30D080047A0C0DAFF7F01000000EA
S30D080047A845250008E920000878
S309080047B0C12000080E
S315080047B400000000EC02002054030020BC03002083
S315080047C400000000000000000000000000000000D7
S315080047D400000000000000000000000000000000C7
S315080047E400000000000000000000000000000000B7
S315080047F400000000000000000000000000000000A7
S315080048040000000000000000000000000000000096
S315080048140000000000000000000000000000000086
S315080048240000000000000000000000000000000076
S315080048340000000000000000000000000000000066
S315080048440000000000000000000000000000000056
S315080048540000000000000000010000000000000045
S315080048640E33CDAB34126DE6ECDE05000B0000000A
S315080048740000000000000000000000000000000026
S315080048840000000000000000000000000000000016
S315080048940000000000000000000000000000000006
S315080048A400000000000000000000000000000000F6
S31508004BD40000000000000000300500200024F40056
S30D08004BE40100000004000000B6
S7050800265D6F
